:100000000C94AC070C94F0070C94F0070C94F007D8
:100010000C94F0070C94F0070C94F0070C94F00784
:100020000C94F0070C94F0070C9412130C94E41346
:100030000C94F0070C94F0070C94F0070C94F00764
:100040000C94F0070C94BC2C0C94F0070C94F00763
:100050000C94F0070C94B4220C94F0070C94F00765
:100060000C94F0070C94F0070C94F0070C94F00734
:100070000C94F0070C94F0070C94F0070C94F00724
:100080000C94F0070C94F0070C94F0070C94F00714
:100090000C94F0070C94F0070C94F0070C94F00704
:1000A0000C94F0070C94F0070C94F007511473149F
:1000B000611573146115B814DB14611530154315FF
:1000C0008A188A18B918B918FD183B19551B551B01
:1000D0005419551B551A551A291B551B551B401BE6
:1000E0000000F0A1F0A329002B000354E1003581AA
:1000F00000001E00140004001D7164004D001F006C
:100100001A0016001B00E1044C0020000800070044
:10011000060050002A0021001500090019004F00B8
:100120004A00220017000A000500000002541908C6
:10013000E3000000E20000002E770608E700000060
:10014000E60000002E7F23001C000B0011000000C1
:100150000454240018000D00100052004B0025002C
:100160000C000E00360051002C00260012000F007B
:100170003700E108280027001300330038713000F1
:100180004E002D002F003482E50031810000010077
:10019000010001000100010000003A0035003100BB
:1001A0000100010001003B00350221026400010052
:1001B0004C003C001E0224062202010001003D000A
:1001C0002D0224022404010001003E00010037003A
:1001D0001104000001000100010000000100000006
:1001E00001000100010000000100000001003F00CB
:1001F00024062402230200000100400022042502FC
:1002000035000100010041002304260235023700B9
:1002100001004200240425041F021E0201004300C5
:1002200031002604310201000100440045000100B4
:100230002D02010000000100010001000100010089
:100240000000010001000100FB00010001000100AD
:100250000100F200F900010001000100F000F100CE
:10026000FA00F400010001000100F300FC00F500B9
:100270000100010001000100F60000000100010082
:100280000100000001000000010001000100000069
:100290000100000001000100010001000100000058
:1002A0000100010001000100A800A90001000100F7
:1002B00001000100AC00AA00B6000100010001002D
:1002C000AB0050000100010001000100520051008C
:1002D0000100AE000100010001004F00000001001C
:1002E0000100010001000100000001000100010007
:1002F00001000100010001000100010001000100F6
:1003000001000100010001000100010001000100E5
:1003100001000100010001000100010001000100D5
:1003200001000000010001000100000001000000C8
:1003300001000100010000000100000001000100B7
:1003400001000100010000000100010001000100A6
:100350000100010001000100010001000100010095
:100360000100010001000100010050000100010036
:1003700001000100520051000100010001000100D4
:1003800001004F0000000100010001000100010018
:100390000000010001000100010001000100010056
:1003A0000100500001000100010001005200510055
:1003B000010001000100010001004F0001000100E7
:1003C0000100010001000100010000000100010026
:1003D0000100000001000000010001000100000018
:1003E0000100000001003F00520051002302000004
:1003F00001004000240021001E00270001004100F0
:10040000250022001F0037000100420026002300C3
:1004100020002700010043003002300024022E009B
:1004200001004400450001000100010000000A0035
:100430002530313662003A200025303258000A72E9
:100440002F63203031323334353637383941424327
:100450004445460A000A002530325800626F756E26
:100460006365213A20006C656674207369646520B9
:1004700061747461636865640A006C6566742073F6
:10048000696465206E6F7420726573706F6E646945
:100490006E670A00747279696E6720746F207265E6
:1004A000736574206D637032333031380A000A444A
:1004B000454255473A20656E61626C65642E0A00BC
:1004C0005B735D004B6579626F6172642073746168
:1004D00072742E0A005B575D005B535D005B525DDA
:1004E000005B445D005B435D0016034500720067DE
:1004F000006F0044006F007800200045005A0000A3
:100500000016034500720067006F0044006F00781A
:1005100000200045005A0000000403090409028D70
:1005200000050100A0FA090400000103010100090F
:100530002111010001223F000705810308000A097B
:100540000401000103010200092111010001224DF3
:10055000000705820308000A0904020001030000E5
:10056000000921110100012236000705830308005C
:100570000A0904030002030000000921110100011F
:100580002220000705840320000107050403200042
:100590000109040400010300000009211101000108
:1005A0002239000705850310000112011001000027
:1005B0000008EDFE07130100010200010501090614
:1005C000A101050719E029E7150025019508750126
:1005D000810205081901290595057501910295010A
:1005E00075039101050719002977150025019578F4
:1005F00075018102C00631FF0974A101097515005A
:1006000025FF9520750881020976150025FF9520A4
:1006100075089102C005010980A10185021601003B
:1006200026B7001A01002AB700751095018100C095
:10063000050C0901A1018503160100269C021A017F
:10064000002A9C02751095018100C005010902A1D4
:10065000010901A1000509190129051500250195C8
:1006600005750181029501750381010501093009B4
:10067000311581257F950275088106093815812578
:100680007F950175088106050C0A38021581257FC2
:10069000950175088106C0C005010906A10105077D
:1006A00019E029E7150025019508750181029501DA
:1006B0007508810105081901290595057501910243
:1006C0009501750391010507190029FF150025FF04
:1006D000950675088100C00A002530325820006B4D
:1006E0006579626F6172645F7265706F72743A20CF
:1006F000000A0025303258006B6579626F617264C0
:100700005F7365745F6C65643A200064656C5F6B51
:1007100065795F6269743A2063616E27742064654D
:100720006C3A20253032580A006164645F6B657949
:100730005F6269743A2063616E2774206164643A71
:1007400020253032580A00646F6E652E0A00626FF1
:100750006F676D61676963207363616E3A202E2E47
:100760002E2000290A002575002F002575005D2820
:10077000002564002000256400200025640020007E
:100780002564007C0025303258006D6F7573656BF1
:100790006579205B62746E7C782079207620685DB4
:1007A000287265702F61636C293A205B006D6B5F66
:1007B000776865656C5F74696D655F746F5F6D61A7
:1007C00078203D2025640A006D6B5F776865656C55
:1007D0005F6D61785F7370656564203D2025640AF4
:1007E000006D6B5F74696D655F746F5F6D6178201C
:1007F0003D2025640A006D6B5F6D61785F737065E5
:100800006564203D2025640A006D6B5F696E746528
:100810007276616C203D2025640A006D6B5F646513
:100820006C6179203D2025640A006D6B5F776865F7
:10083000656C5F74696D655F746F5F6D6178203D95
:100840002025640A006D6B5F776865656C5F6D617C
:10085000785F7370656564203D2025640A006D6BC8
:100860005F74696D655F746F5F6D6178203D2025F1
:10087000640A006D6B5F6D61785F737065656420FD
:100880003D2025640A006D6B5F696E746572766148
:100890006C203D2025640A006D6B5F64656C617996
:1008A000203D2025640A000A00257500363A20778D
:1008B0006865656C5F74696D655F746F5F6D6178A5
:1008C0003A20000A00257500353A20776865656C86
:1008D0005F6D61785F73706565643A20000A00257A
:1008E0007500343A2074696D655F746F5F6D61786F
:1008F0003A20000A00257500333A206D61785F7355
:10090000706565643A20000A00257500323A206956
:100910006E74657276616C286D73293A20000A0046
:10092000257500313A2064656C6179282A31306D73
:1009300073293A20000A092D2056616C75657320D1
:100940002D0A004D3E004D25643E20003F0073659A
:10095000742064656661756C740A00433E200077FC
:10096000686572652064656C74613A2063757273A2
:100970006F723D25642C20776865656C3D25640A9F
:1009800053656520687474703A2F2F656E2E7769F1
:100990006B6970656469612E6F72672F77696B6927
:1009A0002F4D6F7573655F6B6579730A000A092DAA
:1009B000204D6F7573656B6579202D0A4553432F64
:1009C000713A09717569740A313A0964656C617923
:1009D000282A31306D73290A323A09696E746572BA
:1009E00076616C286D73290A333A096D61785F73FB
:1009F000706565640A343A0974696D655F746F5F88
:100A00006D61780A353A09776865656C5F6D617864
:100A10005F73706565640A363A09776865656C5F6F
:100A200074696D655F746F5F6D61780A0A703A0969
:100A30007072696E742076616C7565730A643A0928
:100A40007365742064656661756C74730A75703AB9
:100A5000092B310A646F776E3A092D310A70677578
:100A6000703A092B31300A7067646F776E3A092D3E
:100A700031300A0A7370656564203D2064656C74CA
:100A800061202A206D61785F7370656564202A207B
:100A900028726570656174202F2074696D655F74BC
:100AA0006F5F6D6178290A003F004D3E2000433E94
:100AB00020004C25640A000A092D20436F6E736FD5
:100AC0006C65202D0A4553432F713A09717569747D
:100AD0000A6D3A096D6F7573656B65790A000A09CD
:100AE0002D204D61676963202D0A643A09646562AF
:100AF00075670A783A096465627567206D6174727A
:100B000069780A6B3A096465627567206B6579627A
:100B10006F6172640A6D3A096465627567206D6F72
:100B20007573650A763A0976657273696F6E0A7332
:100B30003A097374617475730A633A09636F6E736B
:100B40006F6C65206D6F64650A302D343A096C61F5
:100B5000796572302D34284631302D4634290A50BB
:100B60006175733A09626F6F746C6F616465720AC4
:100B7000653A09656570726F6D0A6E3A094E4B529F
:100B80004F0A7A3A09736C656570204C45442074AD
:100B90006573740A000A002575002E6E6B726F3A39
:100BA00020000A002575002E737761705F62616313
:100BB0006B736C6173685F6261636B7370616365B3
:100BC0003A20000A002575002E737761705F677206
:100BD0006176655F6573633A20000A002575002E13
:100BE0006E6F5F6775693A20000A002575002E73E5
:100BF0007761705F72616C745F726775693A20002B
:100C00000A002575002E737761705F6C616C745FEC
:100C10006C6775693A20000A002575002E636170C3
:100C2000736C6F636B5F746F5F636F6E74726F6C06
:100C30003A20000A002575002E737761705F636F9C
:100C40006E74726F6C5F636170736C6F636B3A206C
:100C5000000A0025303258006B65796D61705F6362
:100C60006F6E6669672E7261773A20000A002575FB
:100C7000002E6D6F7573653A20000A002575002EF1
:100C80006B6579626F6172643A20000A0025750015
:100C90002E6D61747269783A20000A002575002E65
:100CA000656E61626C653A20000A0025303258009A
:100CB00064656275675F636F6E6669672E726177E0
:100CC0003A20000A0025750064656661756C745FE2
:100CD0006C617965723A20003F004E4B524F3A20CA
:100CE0006F66660A004E4B524F3A206F6E0A0074D0
:100CF000696D65725F636F756E743A202530346C70
:100D0000580A006B6579626F6172645F6E6B726F17
:100D10003A2025580A006B6579626F6172645F69D9
:100D2000646C653A2025580A006B6579626F6172C0
:100D3000645F70726F746F636F6C3A2025580A009D
:100D4000686F73745F6B6579626F6172645F6C6505
:100D5000647328293A2025580A000A092D20537463
:100D600061747573202D0A004743433A20342E39AD
:100D70002E33204156522D4C4942433A20312E38D1
:100D80002E31204156525F415243483A20617672DB
:100D9000350A004F5054494F4E533A204C55464166
:100DA00020424F4F544D41474943204D4F555345E5
:100DB0004B45592045585452414B455920434F4EBD
:100DC000534F4C4520434F4D4D414E44204E4B52C6
:100DD0004F203531320A004255494C443A206130A7
:100DE00038353236352D6469727479202830393AB5
:100DF00034343A3137204A616E2031332032303179
:100E000036290A005649443A203078464545442858
:100E10004572676F446F7820455A29205049443AFB
:100E200020307831333037284572676F446F78202F
:100E3000455A29205645523A203078303030310A10
:100E400000444553433A20742E6D2E6B2E206B6563
:100E500079626F617264206669726D776172652074
:100E6000666F72204572676F646F780A000A092DF9
:100E70002056657273696F6E202D0A000A6D6F75BA
:100E800073653A206F66660A000A6D6F7573653A7E
:100E9000206F6E0A000A6B6579626F6172643A2096
:100EA0006F66660A000A6B6579626F6172643A2048
:100EB0006F6E0A000A6D61747269783A206F666617
:100EC0000A000A6D61747269783A206F6E0A000A2E
:100ED00064656275673A206F6E0A000A6465627520
:100EE000673A206F66660A000A0A626F6F746C6F59
:100EF000616465722E2E2E2000433E2000656563DE
:100F00006F6E6669673A0A00536C656570204C45E0
:100F10004420746573740A000000000000000000A3
:100F2000000000010204060A0F17202C3A4A5D71E6
:100F3000879DB3C7DAE9F5FCFFFCF5E9DAC7B39D95
:100F400087715D4A3A2C20170F0A0604020100003F
:100F5000000000000000000011241FBECFEFDAE007
:100F6000DEBFCDBF04B603FE24C08091F90190918D
:100F7000FA01A091FB01B091FC018730904BA74092
:100F8000B04BB9F41092F9011092FA011092FB01E2
:100F90001092FC0114BE84B7877F84BF88E10FB62E
:100FA000F89480936000109260000FBEE0E0FFE3D1
:100FB000099511E0A0E0B1E0E4E1FDE502C0059093
:100FC0000D92AA33B107D9F711E0AAE3B1E001C04D
:100FD0001D92A93FB107E1F70E944A100C94882E98
:100FE0000C940000FF93EF93E0913A01F0913B01E4
:100FF000309709F00995EF91FF910895FC018591D3
:10100000803011F0EFDFFBCF0895FF27E0E230E200
:1010100047FF0CC0419597FF09C0EDE260957095C0
:1010200080959095611D711D811D911D27FF02C046
:10103000219530E350E2AA27660F771F881F991F7A
:10104000AA1FA41710F0A41B63955A95A9F7AA30FC
:1010500008F0A95FA05DAF93F39561157105810557
:10106000910541F7ED3211F4EF93F395F21718F46F
:101070003F93F395FBCF8F91B5DFFA95E1F7089594
:10108000E991F9918591803021F0853219F0AADF3C
:10109000F9CF089520E0E89455915532C1F35033CB
:1010A00011F4689455915A3348F4505390F3220F39
:1010B000022E220F220F200D250FF4CF0EF42195C2
:1010C00089919991533619F3533729F1533559F1D1
:1010D000BC0188279927E8945C3621F4899199917D
:1010E00068945591543639F446EF7EF077FF0DC081
:1010F0008FEF9FEF0AC055374AE039F0583540E18D
:1011000021F0523642E009F00895FF93EF937DDF1E
:10111000EF91FF91B7CFFF93EF93FC018191803066
:10112000B9F360DFFBCFFF93EF9368DFF1CFDF937D
:10113000CF93CDB7DEB72596A3DFCF91DF9108958A
:1011400061110BC0FC018281882321F085EE0E9491
:10115000271703C085EE0E94EF1780E090E0089506
:1011600008956091BC017091BD018091BE01909184
:10117000BF010E94B72156985E9825982D98269811
:101180002E9827982F98823061F018F4813031F032
:101190000895833049F0843051F00895259A2D9AAE
:1011A0000895269A2E9A0895279A2F9A0895259A97
:1011B0002D9A279A2F9A089581EB98E0892B11F0A8
:1011C0000E94B10880E090E0089556985E982598B6
:1011D0002D9826982E9827982F988FEF90E090932F
:1011E00089008093880090938B0080938A0090936D
:1011F0008D0080938C00259A2D9A2FEF80E792E046
:10120000215080409040E1F700C00000269A2E9ABD
:101210002FEF80E792E0215080409040E1F700C03E
:101220000000279A2F9A2FEF80E792E0215080400C
:101230009040E1F700C0000025982D982FEF80E73F
:1012400092E0215080409040E1F700C000002698D5
:101250002E982FEF80E792E0215080409040E1F7F8
:1012600000C0000027982F9856985E9825982D98D2
:1012700026982E9827982F98089589EA80938000C1
:1012800089E08093810024982C983F988AB18F74CC
:101290008AB96E98479A8BB1806B8BB9769A0E9407
:1012A000E50880EB98E0892B11F00E94B00880E0FF
:1012B00090E0089580E28093000180913C018111CB
:1012C0000EC00E94A90981E080933C012FEF83EDBD
:1012D00090E3215080409040E1F700C0000080E49E
:1012E0000E94AF098093000181112EC00E94D9098C
:1012F00080930001811128C00E94D90980930001C8
:10130000811122C08FE30E94D909809300018111CD
:101310001BC00E94D10980E40E94AF0980930001A4
:10132000811112C08CE00E94D909809300018111C3
:101330000BC00E94D90980930001811105C08FE381
:101340000E94D909809300010E94D1098091000177
:1013500008951092B9008AE08093B800089594EA45
:101360009093BC009091BC0097FFFCCF9091B90086
:10137000987F983021F0903111F081E008958093AA
:10138000BB0084E88093BC008091BC0087FFFCCF49
:101390008091B900887F883111F0803471F780E046
:1013A000089584E98093BC008091BC0084FDFCCF4B
:1013B00008958093BB0084E88093BC008091BC00BA
:1013C00087FFFCCF9091B900987F81E0983209F4B3
:1013D00080E0089584E88093BC008091BC0087FF82
:1013E000FCCF8091BB00089580910001811115C050
:1013F00080E40E94AF098093000181110CC082E15A
:101400000E94D90980930001811105C08FEF0E94CD
:10141000D909809300010E94D10984B1807F84B9E9
:1014200085B1807F85B98AB1837F8AB98BB1837F8B
:101430008BB93E98469808950E945A0980930001FE
:101440000E94F40980B38C7080BB81B3836F81BB31
:10145000AEE3B1E0ECE4F1E08EE08E0F11921D926C
:101460008E13FCCF8DE399E0892B11F00C943D098C
:1014700008959F92AF92BF92CF92DF92EF92FF9228
:101480000F931F93CF93DF93809100018823E1F0A6
:1014900080913D018F5F80933D01811115C084E9EA
:1014A00094E00E94FE070E945A098093000188235D
:1014B00029F08AE794E00E94FE0706C086E694E0E1
:1014C0000E94FE070E94E5080EE311E0C0E0D0E0B4
:1014D000BB24B39482E0A82ECC24C394D12C27E55E
:1014E000E22E24E0F22EC730D10500F580910001F4
:1014F000811164C080E40E94AF09809300018111D2
:1015000012C082E10E94D9098093000181110BC0B1
:10151000C6010C2E01C0880F0A94EAF780950E943C
:10152000D909809300010E94D10948C0CA30A1F0B6
:1015300028F4C83059F0C93061F005C0CC3089F0CA
:1015400070F0CD3089F0209A289810C0219A2998FF
:101550000DC0229A2A980AC0239A2B9807C0529A43
:1015600001C0539A5B9802C03E9A469890EA9A95B9
:10157000F1F79FB1799902C082E001C080E09170DB
:101580009B25982B7C9902C084E001C080E0892BC8
:101590007D9902C038E001C030E0832B7E9902C003
:1015A00020E101C020E0822B9FB19095991F9927DF
:1015B000991F9295990F907E892B10C08091000100
:1015C000811174C080E40E94AF09809300018823D8
:1015D00009F459C0912C0E94D109892DF8019081FC
:1015E000981739F1808380910101882301F180915E
:1015F000D70180FF04C08CE594E00E94FE07809133
:10160000D70180FF0CC0809101011F928F93FF9240
:10161000EF920E9497080F900F900F900F9080917B
:10162000D70180FF04C085E594E00E94FE07A092E8
:1016300001010E94F40921960F5F1F4FCE30D105A2
:1016400009F051CF809101018823B1F0815080933E
:101650000101882339F08FE99FE00197F1F700C07D
:1016600000000AC0ACE4B1E0EEE3F1E0CF01825F3C
:1016700091919D938E13FCCF8CED98E0892BC1F056
:101680000E94DC0815C083E10E94D9098093000103
:101690008111A0CF81E40E94AF09809300018111E4
:1016A00099CF0E94EA09982E909495CF80E096CF2A
:1016B00081E0DF91CF911F910F91FF90EF90DF902C
:1016C000CF90BF90AF909F900895E82FF0E0E45B3B
:1016D000FE4F80810895CF92DF92EF92FF920F9399
:1016E0001F93CF93DF938EE394E00E94FE078CE478
:1016F000E82E81E0F82EC0E0D0E099E3C92E94E016
:10170000D92E00E314E0DF93CF93DF92CF920E94B3
:10171000970886E394E00E94FE07F70181917F011C
:1017200090E00E941D229F938F931F930F930E941E
:1017300097088EE294E00E94FE0721968DB79EB72F
:1017400008960FB6F8949EBF0FBE8DBFCE30D10560
:10175000D1F6DF91CF911F910F91FF90EF90DF9025
:10176000CF9008958B3B910578F4883A910540F528
:10177000853A9105D0F48430910508F0B1C08130EC
:10178000910509F4ADC06BC0803E910508F467C0B7
:10179000883E910508F4A4C09C01205F31092031E6
:1017A000310508F05CC090650895853A910509F40B
:1017B00059C0863A910509F058C082E890E408952E
:1017C000883A910509F454C0893A910509F453C047
:1017D0008A3A910509F452C08B3A910509F451C037
:1017E0008C3A910509F450C08D3A910509F44FC027
:1017F000803B910509F44EC08E3A910509F44DC025
:101800008F3A910509F44CC0813B910509F44BC016
:10181000823B910509F44AC0833B910509F449C014
:10182000843B910509F448C0853B910509F447C004
:10183000863B910509F446C0873B910509F445C0F4
:10184000883B910509F444C0893B910509F443C0E4
:101850008A3B910509F442C080E094E4089580E059
:1018600090E0089581E890E4089583E890E4089575
:1018700082EE94E4089589EE94E408958AEE94E467
:10188000089585EB94E4089586EB94E4089587EB3E
:1018900094E408958CEC94E408958DEC94E4089518
:1018A00083E895E408958AE895E4089582E995E44B
:1018B000089584E995E4089581E296E4089583E229
:1018C00096E4089584E296E4089585E296E4089506
:1018D00086E296E4089587E296E408958AE296E423
:1018E0000895089596E0799FF001112494E5899F69
:1018F000E00DF11D1124E60FF11DEE0FFF1FEA515F
:10190000FF4F859194910895880F991FFC01E05A2B
:10191000F040859194910895880F991FFC01E05241
:10192000FF4F85919491089526E0729FF001112454
:1019300044E5849FE00DF11D1124E60FF11DEE0F2B
:10194000FF1FEA51FF4F859194919C013A95211513
:101950004FE1340708F41EC13F512115304120F4F6
:101960009F700E948C0C08959C01305321153041CA
:1019700018F49927906C0895811520E5920769F471
:101980000E94771B4FEF84E39CE0415080409040E1
:10199000E1F700C000000C94D922813020E59207C5
:1019A00051F48EEA94E00E94FE078091D701816095
:1019B0008093D70108959C0130552115304108F0DE
:1019C00051C0292F33272F70332721303105D9F407
:1019D000AC014370552702C0220F331F4A95E2F72E
:1019E0003C68AC0164E0440F551F6A95E1F7442759
:1019F0005370242B352B73E0880F991F7A95E1F7EC
:101A0000807699271DC02230310529F4982F882728
:101A1000816F906A089523303105A9F4AC014370B9
:101A2000552721E030E002C0220F331F4A95E2F72C
:101A30003C6843E0880F991F4A95E1F7807E9770D4
:101A4000822B932B089524303105E1F4AC014370CF
:101A5000552721E030E002C0220F331F4A95E2F7FC
:101A60003A68E7CF9C0130572115304118F49F7038
:101A7000906208959C0130582115304118F49F70F0
:101A8000906A0895803E9105E0F4803C910558F5F8
:101A90008133910509F46FC048F48932910509F446
:101AA00063C08A32910509F46DC072C08933910513
:101AB000E9F082389105D1F08533910509F44DC0E4
:101AC00067C0833E910581F138F4803E9105B9F0FD
:101AD000823E9105D9F05CC0863E910561F1873E5A
:101AE0009105A1F155C00E94840C08952091EA014E
:101AF00020FD02C021FF4CC080EE90E049C08091E3
:101B0000EA0180FFF9CF89E390E042C08091EA01C9
:101B100082FF0EC08091EA0184FF03C080E090E064
:101B200037C083EE90E034C08091EA0182FFF2CFAB
:101B300082EE90E02DC08091EA0183FF0BC080917E
:101B4000EA0184FDEBCF87EE90E022C08091EA01AC
:101B500083FFF5CF86EE90E01BC08091EA0185FF00
:101B600007C089E290E014C08091EA0185FFF9CFB7
:101B700085E390E00DC08091EA0186FF07C08AE20C
:101B800090E006C08091EA0186FFF9CF81E390E002
:101B90000E94B20B0895089580916D0108959FB73A
:101BA000F89410925C019FBF9091F001943009F07D
:101BB00057C09091E9009F703091EC00232F217065
:101BC00030FD20E8922B24E02093E9002091EB00E7
:101BD00020FF43C02091EE0027FF3FC020915A0113
:101BE000222321F02091E80025FF37C010925A01EE
:101BF00026E03091E80035FD15C03091F001343019
:101C000061F53091EB0035FD28C0215021F481E0D1
:101C100080935A0122C0EFE9FFE03197F1F700C04D
:101C20000000E7CF8093F1008091E80085FD0AC0B5
:101C30008091E80080FFFCCF8091E8008E77809350
:101C4000E80006C08FB7F89421E020935C018FBFB5
:101C50009F709093E90080E008959F709093E90051
:101C60008FEF0895CF93DF9300D01F92CDB7DEB7EB
:101C70009C018091F001843019F593E099833B83B6
:101C80002A839093E9008FEF9091E800815095FDB1
:101C900006C095ED9A95F1F700008111F5CF80917E
:101CA000E80085FF0DC040E050E063E070E0CE0149
:101CB00001960E9402118091E8008E778093E800DF
:101CC0000F900F900F90DF91CF910895CF93DF93F6
:101CD00000D01F92CDB7DEB72091F001243021F55E
:101CE00022E029839B838A8383E08093E9008FEF3E
:101CF0009091E800815095FD06C095ED9A95F1F719
:101D000000008111F5CF8091E80085FF0DC040E013
:101D100050E063E070E0CE0101960E9402118091D4
:101D2000E8008E778093E8000F900F900F90DF917E
:101D3000CF9108952091F0012430F1F422E0209316
:101D4000E9002FEF3091E800215035FD06C035ED58
:101D50003A95F1F700002111F5CF2091E80025FF19
:101D60000BC040E050E065E070E00E9402118091FD
:101D7000E8008E778093E8000895CF93DF93209159
:101D8000F001243009F048C0EC0180910C01882357
:101D9000E1F080910D018823C1F085E08093E90096
:101DA0008FEF9091E800815095FD06C095E19A95DE
:101DB000F1F700008111F5CF8091E80085FF2CC07C
:101DC00040E050E060E170E017C081E08093E900FE
:101DD0008FEF9091E800815095FD06C095ED9A95A2
:101DE000F1F700008111F5CF8091E80085FF14C064
:101DF00040E050E068E070E0CE010E940211809166
:101E0000E8008E778093E80080E1FE01ADE5B1E067
:101E100001900D928A95E1F7DF91CF91089585EEBB
:101E200094E00E94FE078091EF01811109C00E9499
:101E300097120E94F4128091E20084608093E20085
:101E4000089581EE94E00E94FE071092EF0108953C
:101E50008DED94E00C94FE0789ED94E00E94FE075E
:101E60000C94A92C85ED94E00E94FE070E94732239
:101E70000E94AF2C0E9499150C94CB0D20915B0110
:101E80002F5F822F62E30E941D2E992319F0209369
:101E90005B01089510925B0180915C01882371F1D0
:101EA0008091F001843041F58091E9008F7020919C
:101EB000EC00922F917020FD90E8892B94E0909394
:101EC000E9009091EB0090FF14C09091EE0097FF15
:101ED00010C09091E80095FF03C01092F100F9CF77
:101EE0009091E80090FF05C09091E8009E77909354
:101EF000E8008F708093E90010925C01089542E041
:101F000061EC81E00E94111242E061EC82E00E94EB
:101F1000111242E061EC83E00E94111242E261EC96
:101F200084E00E94111242E161EC85E00C941112F0
:101F30008091F201833009F455C030F4813071F0A2
:101F4000823009F48EC008958A3009F47AC08B304B
:101F500009F460C0893009F09CC020C08091F10173
:101F6000813A09F096C08091E800877F8093E8006D
:101F70008091F5019091F601892B21F460E18DE5C6
:101F800091E003C060E080E090E070E00E944D11BD
:101F90008091E8008B778093E80008958091F101AB
:101FA000813209F076C08091F5019091F601009799
:101FB00019F0049709F06DC08091E800877F809345
:101FC000E8008091E80082FD05C08091F001811158
:101FD000F8CF5FC08091F10080936D018091E8009F
:101FE0008B7753C08091F101813A09F052C0809102
:101FF000F5019091F601892B09F04BC08091E80022
:10200000877F8093E8008091E80080FFFCCF80917B
:102010000C0136C08091F1018132D9F58091F50132
:102020009091F601892BA9F58091E800877F809334
:10203000E8000E9446128091F30180930C010C94F9
:10204000771B8091F101813221F58091E800877F33
:102050008093E8000E9446128091F40180936E0103
:1020600008958091F101813AA1F48091E800877F81
:102070008093E8008091E80080FFFCCF80916E01A2
:102080008093F1008091E8008E778093E8000C94B3
:102090004612089584B7877F84BF88E10FB6F8940D
:1020A00080936000109260000FBE90E080E80FB651
:1020B000F89480936100909361000FBE0E942616F1
:1020C0000E9497120E94F4128091E2008460809333
:1020D000E2008FEC9DE00E94B22178940E94791575
:1020E0000E94281682E091E00E9494150E94972C8D
:1020F00084EC94E00E94FE078091F001853089F421
:1021000080EC94E00E94FE070E9437228091EE014D
:10211000882391F30E945F22882371F30E94EC10C0
:10212000EBCF0E945616E8CF292F332723303105F5
:10213000C9F064F42130310581F02230310509F015
:1021400043C08DE890E02DE135E042C021323105F9
:10215000F1F02232310541F137C082E190E02AEA04
:1021600035E036C099278130910541F082309105E4
:1021700041F0892B49F5E9E1F5E005C0E1E0F5E042
:1021800002C0E9EEF4E0849190E09F0121C0653047
:10219000D8F4E62FF0E0EE0FFF1FEB5DFE4F20813D
:1021A000318189E090E014C0653070F470E0FB018B
:1021B000EE0FFF1FE55EFE4F20813181FB01EA5EDD
:1021C000FE4F808190E004C080E090E020E030E0AD
:1021D000FA0131832083089580E189BD82E189BDC0
:1021E00009B400FEFDCF8091D8008F7D8093D80088
:1021F0008091E00082608093E0008091E00081FDAA
:10220000FCCF0895CF92DF92EF92FF920F931F932E
:10221000CF93DF93EC018B016A010E94651281115B
:1022200033C0C114D10439F0F60180819181081BBB
:10223000190BC80FD91FE12CF12C0115110519F14B
:102240008091E80085FD16C08091E8008E7780932C
:10225000E800C114D10449F0F60180819181E80EB3
:10226000F91EF182E08285E00FC00E94651288238A
:1022700021F30AC089918093F10001501109FFEF09
:10228000EF1AFF0ADACF80E0DF91CF911F910F9113
:10229000FF90EF90DF90CF9008952091F70130915B
:1022A000F8012617370748F06115710539F42091B8
:1022B000E8002E772093E80001C0B90140E06115E5
:1022C0007105A9F12091F001222309F443C02530C2
:1022D00009F442C02091E80023FD40C02091E800AD
:1022E00022FD32C02091E80020FFE9CF4091F300A9
:1022F0002091F20030E0342BFC01CF016115710513
:1023000059F02830310540F481918093F1006150FB
:1023100071092F5F3F4FF1CF41E02830310509F0BF
:1023200040E02091E8002E772093E800C8CF4111CB
:10233000C9CF0AC08091F001882361F0853061F037
:102340008091E80083FD0AC08091E80082FFF2CF0F
:1023500080E0089582E0089583E0089581E0089583
:102360002091F7013091F8012617370748F06115E1
:10237000710539F42091E8002E772093E80001C020
:10238000B901FC0120E06115710591F18091F00126
:10239000882309F440C0853009F43FC08091E800EB
:1023A00083FD3DC08091E80082FD2FC08091E80050
:1023B00080FFE9CF2091F3008091F20090E0922B12
:1023C0006115710559F08830910540F424912093EE
:1023D000F1003196615071090196F2CF21E0089722
:1023E00009F020E08091E8008E778093E800CBCF61
:1023F0002111CCCF0AC08091F001882361F0853093
:1024000061F08091E80083FD0AC08091E80082FFBE
:10241000F2CF80E0089582E0089583E0089581E09E
:102420000895982F973058F59093E900981739F050
:102430007091EC002091ED005091F00003C0242F2A
:10244000762F50E021FF19C03091EB003E7F309392
:10245000EB003091ED003D7F3093ED003091EB00CB
:1024600031603093EB007093EC002093ED005093BB
:10247000F0002091EE0027FF07C09F5FD3CF8F7041
:102480008093E90081E0089580E008958091F10152
:1024900087FF11C08091E80082FD05C08091F001A6
:1024A0008111F8CF11C08091E8008B770BC080912B
:1024B000F001882349F08091E80080FFF8CF8091F7
:1024C000E8008E778093E80008952091E400309131
:1024D000E50095E64091EC00842F817040FF22C01A
:1024E0008091E80080FD1CC08091F001882391F06C
:1024F000853091F08091EB0085FD10C04091E400A3
:102500005091E5004217530729F39A01915011F7B2
:1025100084E0089582E0089583E0089581E00895BD
:1025200080E008954091E80042FFDECF08950E94C8
:1025300005130E940D13E0EEF0E08081816080833E
:10254000E8EDF0E080818F77808319BCA7EDB0E0E3
:102550008C918E7F8C9380818F7E80831092EF018F
:1025600008950F931F93CF93DF930E9405130E944A
:102570000D13C8EDD0E088818F77888388818068CB
:10258000888388818F7D888319BC1092F001109216
:10259000EC011092EE011092ED0100EE10E0F80156
:1025A00080818B7F808388818160888342E060E0C6
:1025B00080E00E941112E1EEF0E080818E7F808346
:1025C000E2EEF0E08081816080838081886080839A
:1025D000F80180818E7F8083888180618883DF918C
:1025E000CF911F910F910895E8EDF0E080818F7EEB
:1025F0008083E7EDF0E080818160808384E082BFAA
:1026000081E08093EF010C94B112E8EDF0E080815D
:102610008E7F80831092E20008951092DA0010926B
:10262000E10008951F920F920FB60F9211242F937D
:102630003F934F935F936F937F938F939F93AF934A
:10264000BF93EF93FF938091E10082FF0BC08091D5
:10265000E20082FF07C08091E1008B7F8093E10060
:102660000E943E0F8091DA0080FF1FC08091D80049
:1026700080FF1BC08091DA008E7F8093DA0080910A
:10268000D90080FF0DC080E189BD82E189BD09B418
:1026900000FEFDCF81E08093F0010E940F0F05C086
:1026A00019BC1092F0010E94210F8091E10080FF7F
:1026B00019C08091E20080FF15C08091E2008E7FFA
:1026C0008093E2008091E20080618093E20080913B
:1026D000D80080628093D80019BC85E08093F00117
:1026E0000E942C0F8091E10084FF30C08091E200B5
:1026F00084FF2CC080E189BD82E189BD09B400FE60
:10270000FDCF8091D8008F7D8093D8008091E1002B
:102710008F7E8093E1008091E2008F7E8093E200C3
:102720008091E20081608093E2008091EC01882337
:1027300011F084E007C08091E30087FD02C081E0D2
:1027400001C083E08093F0010E94320F8091E1008C
:1027500083FF29C08091E20083FF25C08091E100C2
:10276000877F8093E10082E08093F0011092EC017A
:102770008091E1008E7F8093E1008091E2008E7F66
:102780008093E2008091E20080618093E20042E069
:1027900060E080E00E9411128091F00088608093D8
:1027A000F0000E94280FFF91EF91BF91AF919F9190
:1027B0008F917F916F915F914F913F912F910F90EA
:1027C0000FBE0F901F9018951F920F920FB60F9289
:1027D00011242F933F934F935F936F937F938F9326
:1027E0009F93AF93BF93CF93DF93EF93FF93C091EA
:1027F000E900CF708091EC00D82FD17080FDD0E837
:102800001092E9008091F000877F8093F000789427
:102810000E9428141092E9008091F0008860809353
:10282000F000CD2BCF70C093E900FF91EF91DF91C5
:10283000CF91BF91AF919F918F917F916F915F9158
:102840004F913F912F910F900FBE0F901F901895B1
:102850001F93CF93DF93CDB7DEB7AA970FB6F89447
:10286000DEBF0FBECDBFE1EFF1E088E08E0F9091AB
:10287000F10091938E13FBCF0E94980F8091E80096
:1028800083FF1FC18091F1019091F201492F50E027
:102890004A30510508F015C1FA01EA5AFF4F0C946D
:1028A0003D2E803881F0823809F00BC18091F5010E
:1028B0008F708093E9008091EB0085FB882780F979
:1028C0001092E90006C08091ED019091EE01911106
:1028D00082609091E800977F9093E8008093F100E8
:1028E0001092F100C8C0282F2D7F09F0EAC088237C
:1028F00019F0823061F0E5C08091F301813009F078
:10290000E0C0933009F080E08093EE012BC080910D
:10291000F301811127C08091F5018F7009F4D1C0B6
:102920008093E9002091EB0020FF1CC0933021F43C
:102930008091EB00806214C09091EB0090619093C5
:10294000EB0021E030E0A90102C0440F551F8A9539
:10295000E2F74093EA001092EA008091EB00886071
:102960008093EB001092E9008091E800877F86C099
:102970008111A7C01091F3011F778091E300807847
:10298000812B8093E3008091E800877F8093E800AB
:102990000E9446128091E80080FFFCCF8091E30006
:1029A00080688093E300111102C082E001C083E0DF
:1029B0008093F00186C08058823008F082C08091F8
:1029C000F3019091F4018C3D53E0950779F583E094
:1029D0008A838AE289834FB7F894DE01139620E058
:1029E0003EE051E2E32FF0E050935700E49120FFE6
:1029F00003C0E295EF703F5FEF708E2F90E0EA30FA
:102A000010F0C79601C0C0968D939D932F5F24311F
:102A100049F74FBF8091E800877F8093E8006AE222
:102A200070E0CE0101960E944D1114C0AE014F5FBF
:102A30005F4F6091F5010E949410BC01892B09F44D
:102A400040C09091E800977F9093E80089819A8137
:102A50000E94B0118091E8008B778093E80031C02C
:102A6000803879F58091E800877F8093E800809135
:102A7000EC018093F1008091E8008E778093E8006C
:102A80000E9446121EC081111CC09091F301923029
:102A9000C0F48091E800877F8093E8009093EC0178
:102AA0000E9446128091EC01811106C08091E300E2
:102AB00087FD02C081E001C084E08093F0010E94A4
:102AC0007F0F8091E80083FF0AC08091E800877F34
:102AD0008093E8008091EB0080628093EB00AA96DF
:102AE0000FB6F894DEBF0FBECDBFDF91CF911F911F
:102AF0000895CF938091F0018823A1F0C091E9005F
:102B0000CF709091EC00892F817090FD80E8C82BE8
:102B10001092E9008091E80083FD0E942814CF7094
:102B2000C093E900CF91089590937401809373014D
:102B30000895E0917301F0917401309721F00190B4
:102B4000F081E02D099480E00895EF92FF920F93B9
:102B50001F93CF93DF93E0917301F091740130974D
:102B6000B1F18C010280F381E02D09958091D701AC
:102B700082FF2DC080FF04C08FED96E00E94FE070B
:102B8000E80110E189EDE82E86E0F82E8091D7016A
:102B900080FF0BC088811F928F93FF92EF920E945B
:102BA00097080F900F900F900F90115021961111D0
:102BB000EDCF8091D70180FF0AC087ED96E0DF91CD
:102BC000CF911F910F91FF90EF900C94FE07DF9132
:102BD000CF911F910F91FF90EF900895E0917301B5
:102BE000F0917401309721F00480F581E02D099473
:102BF000089520917101309172018217930771F04D
:102C00009093720180937101E0917301F0917401CE
:102C1000309721F00680F781E02D099408952091E6
:102C20006F01309170018217930771F090937001DA
:102C300080936F01E0917301F0917401309721F05E
:102C40000084F185E02D0994089508950C942516CB
:102C50000E9475220E941C0A0C943B23CF93C82F1C
:102C60008091D70182FF1EC080FF04C088EF96E0EC
:102C70000E94FE078091D70180FF0CC01F92CF9366
:102C800083EF96E09F938F930E9497080F900F9089
:102C90000F900F908091D70180FF04C081EF96E0E4
:102CA0000E94FE078C2FCF910C94CB0DCF92DF9218
:102CB000EF92FF920F931F93CF93DF93CDB7DEB7C1
:102CC0002B970FB6F894DEBF0FBECDBF0E94390A16
:102CD00086E7C82E81E0D82E00E010E0E02E802F9D
:102CE0000E94650BF60141916F01F42EF826B1F4B4
:102CF0000F5F1F4F0E30110589F78FEF89838A838D
:102D00001B820E947E228160782F9D838C83498163
:102D10005A816B818D810E94F91640C09091D70134
:102D200091FF04C08B870E946B0B8B8520E030E005
:102D30004F2D50E0922FBA01022E02C07595679573
:102D40000A94E2F760FF24C02E83EF8221E030E096
:102D5000690102C0CC0CDD1C9A95E2F790E08C2151
:102D60009D21892B09F420E028870E947E22816022
:102D7000782F9A8789874E815F8168858A850E942E
:102D8000F916F801EA58FE4F8081C826C08206C0B5
:102D90002F5F3F4F2630310569F6AACF0E94AC263F
:102DA000109175010E9499151817A1F00E949915AC
:102DB000809375012B960FB6F894DEBF0FBECDBF82
:102DC000DF91CF911F910F91FF90EF90DF90CF9007
:102DD0000C942E162B960FB6F894DEBF0FBECDBF07
:102DE000DF91CF911F910F91FF90EF90DF90CF90E7
:102DF0000895CF93DF93CDB7DEB72B970FB6F89436
:102E0000DEBF0FBECDBF4F83588769877A878B8718
:102E1000DE01119686E0FD0111928A95E9F785E0C1
:102E2000FE01379601900D928A95E1F749815A810A
:102E30006B817C818D819E810E94111E2B960FB625
:102E4000F894DEBF0FBECDBFDF91CF910895CF9331
:102E5000882309F4C2C0C82F823859F40E949915FA
:102E600081FDBBC089E30E94AD200E948C2189E3D3
:102E70000CC0833879F40E94991580FDAEC083E5BB
:102E80000E94AD200E948C2183E50E940021CF91F9
:102E90000C948C21843859F40E94991582FD9DC0B0
:102EA00087E40E94AD200E948C2187E4EECF8CEF56
:102EB0008C0F813A48F48C2F0E943F2B81118DC0DA
:102EC0008C2F0E94AD20E3CF80E28C0F883048F435
:102ED000C77081E001C0880FCA95EAF70E945521AA
:102EE000D6CF8BE58C0F833078F4C53A29F0C63AFB
:102EF00031F083E890E005C081E890E002C082E80C
:102F000090E0CF910C94F91588E58C0F833108F08F
:102F100064C0C83A39F1C93A41F1CA3A49F1CB3AE9
:102F200051F1CC3A59F1CD3A61F1C03B69F1CE3A59
:102F300071F1CF3A79F1C13B81F1C23B89F1C33BD9
:102F400091F1C43B99F1C53BA1F1C63BA9F1C73B47
:102F5000B1F1C83BB9F1C93BC1F1CA3BC9F180E04D
:102F600090E038C082EE90E035C089EE90E032C04B
:102F70008AEE90E02FC085EB90E02CC086EB90E0CD
:102F800029C087EB90E026C08CEC90E023C08DEC4C
:102F900090E020C083E891E01DC08AE891E01AC06B
:102FA00082E991E017C084E991E014C081E292E0E7
:102FB00011C083E292E00EC084E292E00BC085E291
:102FC00092E008C086E292E005C087E292E002C08B
:102FD0008AE292E0CF910C940F16CF910895882346
:102FE00009F44BC0823859F40E94991581FF45C0FD
:102FF00089E30E94AD200E948C2189E30CC08338B4
:1030000071F40E94991580FF38C083E50E94AD20BD
:103010000E948C2183E50E9400210C948C2184382D
:1030200059F40E94991582FF28C087E40E94AD20C0
:103030000E948C2187E4EFCF9CEF980F913A58F3D0
:1030400090E2980F983050F4877091E001C0990F8A
:103050008A95EAF7892F0E945B21DFCF9BE5980FC5
:10306000933020F480E090E00C94F915885A833175
:1030700020F480E090E00C940F160895882321F04E
:103080000E9455210C948C210895882321F00E94E0
:103090005B210C948C210895BF92CF92DF92EF9226
:1030A000FF920F931F93CF93DF9300D000D000D0F7
:1030B000CDB7DEB725E0FC01DE01119601900D923F
:1030C0002A95E1F7FC014081318102812581229519
:1030D0002F7063817481672B09F4E7C23F3F19F4B5
:1030E0004F3F09F4E2C27C0149833A8389819A8186
:1030F0002E830E946C20182FB92E0E946B200E94F4
:10310000321FEB2DE295EF70F0E0E05AFF4F2E8179
:103110000C943D2E8B2D807F9B2D9F70F92E882344
:1031200019F0F29480EFF822002349F0FF2009F40F
:1031300069C28F2D0E9465210E948C2163C2812F5C
:103140000E94EF17FF2009F4B0C28F2D0E946B215F
:1031500026960FB6F894DEBF0FBECDBFDF91CF919C
:103160001F910F91FF90EF90DF90CF90BF900C9444
:103170008C213B2D307F8B2D8F70303211F082955A
:10318000807F112319F0113021F12DC00023B9F0F7
:10319000222309F4A1C1213009F09EC126960FB661
:1031A000F894DEBF0FBECDBFDF91CF911F910F917D
:1031B000FF90EF90DF90CF90BF900C947521222369
:1031C00019F0213009F471C28E830E9478218E811A
:1031D00097C1002321F0263008F067C27DC1253059
:1031E00008F063C28DC1002321F0222309F474C1C9
:1031F00009C2222309F484C11AC22B2D26952695D3
:10320000237030E02115310521F021303105D1F056
:103210004CC2002321F0812F9B2D937002C080E0CF
:1032200090E026960FB6F894DEBF0FBECDBFDF91BB
:10323000CF911F910F91FF90EF90DF90CF90BF90B3
:103240000C94F915002321F0812F9B2D937002C05F
:1032500080E090E026960FB6F894DEBF0FBECDBF9B
:10326000DF91CF911F910F91FF90EF90DF90CF9062
:10327000BF900C940F16812F002319F00E94322565
:1032800002C00E949A2526960FB6F894DEBF0FBEA4
:10329000CDBFDF91CF911F910F91FF90EF90DF9005
:1032A000CF90BF900C941F268B2D837009F07BC0AC
:1032B0000111FBC1812F829586958770880F880F39
:1032C000912F9F70C92ED12CE12CF12C082E04C017
:1032D000CC0CDD1CEE1CFF1C0A94D2F714FF12C0AC
:1032E0004FE050E060E070E004C0440F551F661FDF
:1032F000771F8A95D2F7CB01BA01609570958095BA
:10330000909503C060E070E0CB012B2D26952695AB
:103310002370422F50E042305105D9F0433051051F
:1033200069F16C297D298E299F294130510551F180
:1033300026960FB6F894DEBF0FBECDBFDF91CF91BA
:103340001F910F91FF90EF90DF90CF90BF900C9462
:10335000591F6C297D298E299F2926960FB6F8942E
:10336000DEBF0FBECDBFDF91CF911F910F91FF90B8
:10337000EF90DF90CF90BF900C94751F0E94591F63
:10338000C701B60126960FB6F894DEBF0FBECDBFBB
:10339000DF91CF911F910F91FF90EF90DF90CF9031
:1033A000BF900C943D1F002319F08B2D817001C03C
:1033B0008695882309F479C1812F82958695877037
:1033C000880F880F912F9F70C92ED12CE12CF12CE2
:1033D000082E04C0CC0CDD1CEE1CFF1C0A94D2F796
:1033E00014FF12C04FE050E060E070E004C0440FF2
:1033F000551F661F771F8A95D2F7CB01BA016095DA
:1034000070958095909503C060E070E0CB012B2D06
:10341000269526952370422F50E042305105D9F071
:103420004330510569F16C297D298E299F2941304E
:10343000510551F126960FB6F894DEBF0FBECDBFF1
:10344000DF91CF911F910F91FF90EF90DF90CF9080
:10345000BF900C9433206C297D298E299F292696B4
:103460000FB6F894DEBF0FBECDBFDF91CF911F9195
:103470000F91FF90EF90DF90CF90BF900C944F2072
:103480000E943320C701B60126960FB6F894DEBF1E
:103490000FBECDBFDF91CF911F910F91FF90EF90A5
:1034A000DF90CF90BF900C941720103FD1F118F40B
:1034B000103E50F4A2C0123F09F464C008F44DC09D
:1034C000133F09F474C099C01F708B2D8F710023B6
:1034D000A1F00E94B01F812F26960FB6F894DEBF90
:1034E0000FBECDBFDF91CF911F910F91FF90EF9055
:1034F000DF90CF90BF900C943E180E94D11F812F77
:1035000026960FB6F894DEBF0FBECDBFDF91CF91E8
:103510001F910F91FF90EF90DF90CF90BF900C9490
:1035200045180023B1F0253008F0BFC08B2D8F71F6
:1035300026960FB6F894DEBF0FBECDBFDF91CF91B8
:103540001F910F91FF90EF90DF90CF90BF900C9460
:10355000F61F263008F0A9C0E9CF0023A9F08B2D73
:103560008F7126960FB6F894DEBF0FBECDBFDF91E8
:10357000CF911F910F91FF90EF90DF90CF90BF9070
:103580000C94B01F002359F38B2D8F7126960FB624
:10359000F894DEBF0FBECDBFDF91CF911F910F9189
:1035A000FF90EF90DF90CF90BF900C94D11F00233D
:1035B00099F08B2D8F7126960FB6F894DEBF0FBE53
:1035C000CDBFDF91CF911F910F91FF90EF90DF90D2
:1035D000CF90BF900C949B1F26960FB6F894DEBF39
:1035E0000FBECDBFDF91CF911F910F91FF90EF9054
:1035F000DF90CF90BF900C94911F0023A9F022235D
:1036000009F4ADCF812F26960FB6F894DEBF0FBE1A
:10361000CDBFDF91CF911F910F91FF90EF90DF9081
:10362000CF90BF900C942717222309F4ADCF812FA0
:1036300026960FB6F894DEBF0FBECDBFDF91CF91B7
:103640001F910F91FF90EF90DF90CF90BF900C945F
:10365000EF174B2D4F70612FC7010E94A0082696CF
:103660000FB6F894DEBF0FBECDBFDF91CF911F9193
:103670000F91FF90EF90DF90CF90BF900C94B51E0C
:103680004B2D4F70612FC70126960FB6F894DEBF01
:103690000FBECDBFDF91CF911F910F91FF90EF90A3
:1036A000DF90CF90BF900C94710C26960FB6F894D3
:1036B000DEBF0FBECDBFDF91CF911F910F91FF9065
:1036C000EF90DF90CF90BF9008950E9472210E94EA
:1036D00047210E948C210E9452270E941F2680E0D1
:1036E00090E00E94F91580E090E00C940F160E9483
:1036F00062210C94651B0E946C20292F22952F704B
:1037000030E02C3031054CF42A3031056CF4225075
:1037100031092230310588F407C02C30310549F0D9
:103720002F30310531F009C0803E48F0803F29F448
:1037300006C093FB882780F9089580E0089581E012
:103740000895CF93DF9300D000D01F92CDB7DEB79E
:103750000F900F900F900F900F90DF91CF910895E1
:10376000CF93DF9300D000D000D0CDB7DEB7269640
:103770000FB6F894DEBF0FBECDBFDF91CF91089595
:103780001F93CF93DF93C091840116E08091850150
:10379000C81799F0D0E01C9FF0011D9FF00D112477
:1037A000EA57FE4F40815181628173818481958106
:1037B0000E94B01B2196C770E9CFDF91CF911F9176
:1037C00008954091B6015091B7016091B801709190
:1037D000B9018091BA019091BB010C94B01B80910A
:1037E000BB0182958F7009F054C08091B801882385
:1037F00009F44FC080918401A09185016091B601C8
:103800007091B7014091B9015091BA01B6E08A17A1
:1038100009F43FC090E041155105C1F17F3F11F41B
:103820006F3FA1F1B89FF001B99FF00D1124EA5745
:10383000FE4F218172132AC02081621327C022818A
:10384000211124C0238134812417350710F421501D
:103850003109241B350B283C3105C0F42091BB01F4
:103860002F7020612093BB0126E0289FF001299F43
:10387000F00D1124E557FE4F80818F7080618083A9
:1038800086EB91E00E944C180C94C01B0196877047
:10389000BECF0895CF92DF92EF92FF920F931F93C6
:1038A000CF93DF93CDB7DEB762970FB6F894DEBF44
:1038B0000FBECDBF8C0185E0F801DE011D960190A1
:1038C0000D928A95E1F7D8014C9111965C91119770
:1038D00012966C9112971396CD90DC9014973091BC
:1038E000B6017091B7018091B9019091BA0100972A
:1038F00009F46BC17F3F19F43F3F09F466C1E090C2
:10390000B801EE2009F4C0C02091BB01C816D90649
:1039100028F0F601E81BF90BCF0104C080959095C3
:103920008C0D9D1DFF24F394883C910578F0F12CBB
:10393000207F09F0C6C07C2DD98AC88A89890E9457
:10394000A11B86EB91E00E944C18B1C0822F807FB2
:1039500009F046C0751314C0341312C0611110C0B1
:103960002F7020612093BB010E94E11B86EB91E048
:103970000E944C188091BB01D80115968C932EC0E3
:10398000CD2819F15F3F11F44F3FF9F0F62E611188
:103990001CC0809184012091850136E0821709F4D2
:1039A0005AC090E0389FF001399FF00D1124EA577A
:1039B000FE4F7181571306C07081471303C0728197
:1039C000711103C001968770E9CFF62E662309F4C2
:1039D00018C18091BB0181608093BB01F12C11C1A2
:1039E000751308C0341306C0611104C08091BB0177
:1039F000D801C3C04D875E878D859E856A8B0E94E6
:103A00007B1B6A898823E1F16623D1F12091BB01F8
:103A1000822F82958F7090E0029774F08091B601AA
:103A20009091B70198878F831986DB86CA862C8789
:103A3000CE0107960E944C1886E0F801A6EBB1E093
:103A400001900D928A95E1F70E94EF1B0E94E11B05
:103A5000FF24F394D6C04D875E878D859E850E9496
:103A60006C20292F22952F7030E0223031050CF088
:103A7000BCC09F7009F0B6C0805E883008F4C1C039
:103A8000C8010E944C18E4CFC816D90608F453C0E8
:103A9000F601E81BF90BCF01883C910508F450C0F2
:103AA000F12C7C2DD98AC88A89890E94A11BE6EB5A
:103AB000F1E086E0DF011D928A95E9F70E94E11BA3
:103AC000A0C0751314C0341312C0611110C08091CE
:103AD000BB01F8018583C8010E944C1886E0E6EB23
:103AE000F1E0DF011D928A95E9F7FE2C8AC04D872F
:103AF0005E878D859E856A8B0E947B1B6A898823E1
:103B000009F4BECF662309F4BBCF2091BB01822FFD
:103B100082958F7090E002970CF48ECF8091B60161
:103B20009091B7019A8389831B82DD82CC822E8398
:103B3000CE0101967FCF809590958C0D9D1DACCFC9
:103B4000F62E662309F49CCF75132EC034132CC0B7
:103B50002091BB0120FD1FC0822F82958F70D9F06C
:103B6000D80115962C9315978F3049F08F5F982FB9
:103B70009295907F822F8F70892B15968C93C80118
:103B80000E944C1886E0F801A6EBB1E001900D927E
:103B90008A95E1F793CF86E0F801A6EBB1E00190BA
:103BA0000D928A95E1F72DC04D875E878D859E85A4
:103BB0000E947B1B811140CF8091BB01816080936B
:103BC000BB01C8010E944C181CC0662309F458CFE1
:103BD0004D875E878D859E850E947B1B882309F417
:103BE0004FCF2ACF811148CF0CC0243031050CF0C3
:103BF00047CF9F7009F440CFF8019581907F09F07D
:103C00003BCF8F2D62960FB6F894DEBF0FBECDBFAF
:103C1000DF91CF911F910F91FF90EF90DF90CF90A8
:103C200008951F93CF93DF93CDB7DEB72C970FB6D0
:103C3000F894DEBF0FBECDBF4F83588769877A8760
:103C40008B879C87CE0107960E944A1C882369F0C7
:103C50008F8198852A853B85232BF1F19F3F09F0C1
:103C600063C08F3F09F060C037C086E0FE01379621
:103C7000DE01119601900D928A95E1F76F817885AA
:103C8000EA85FB85309741F17F3F11F46F3F21F1C9
:103C90002091850130E0C9010196877099274091F4
:103CA000840150E08417950709F447C069837A833B
:103CB000FD83EC8396E0929FD001939FB00D112479
:103CC000AA57BE4FFE01319601900D929A95E1F7E9
:103CD000809385010E94C01B16E080918401909121
:103CE00085018917C1F1189FC00111248A579E4F81
:103CF0000E944A1C882379F1E09184011E9FF00103
:103D00001124EA57FE4F4081518162817381848181
:103D100095810E94B01B8091840190E0019687708C
:103D2000992780938401D9CF4F81588569857A85F9
:103D30008B859C850E94B01BCFCF0E94771B109271
:103D4000850110928401E6EBF1E086E0DF011D922F
:103D50008A95E9F7C1CF2C960FB6F894DEBF0FBE57
:103D6000CDBFDF91CF911F910895EF92FF920F93F6
:103D70001F93CF93DF938C01892B09F46CC0F12C36
:103D8000EE24E394E8012196F8018491843740F40D
:103D9000843008F051C0813081F0823019F15BC06D
:103DA000853709F444C0A8F19CE7980F903708F0D4
:103DB00052C08F770E94EF1741C00E5F1F4FFE0168
:103DC000C49180E28C0F883048F4C7708E2D01C0FA
:103DD000880FCA95EAF70E94652114C08C2F0E94B3
:103DE00027172DC00E5F1F4FFE01C49180E28C0F7C
:103DF000883058F4C7708E2D01C0880FCA95EAF735
:103E00000E946B210E948C211AC08C2F0E94EF17F8
:103E100016C00E5F1F4FFE01C491CC2381F08FE9C5
:103E20009FE00197F1F700C00000C150F6CF0E5F90
:103E30001F4FFE01F49003C00E9427178E018F2DA3
:103E4000882309F49FCFEFE9FFE03197F1F700C035
:103E500000008150F5CFDF91CF911F910F91FF901E
:103E6000EF90089508956093C0017093C10180930D
:103E7000C2019093C3010C94651B0F931F93009193
:103E8000C0011091C1012091C2013091C301DC0138
:103E9000CB01802B912BA22BB32B8093C00190934D
:103EA000C101A093C201B093C3011F910F910C9463
:103EB000651B0F931F930091C0011091C1012091C8
:103EC000C2013091C301DC01CB0180239123A223E5
:103ED000B3238093C0019093C101A093C201B0931A
:103EE000C3011F910F910C94651B0F931F930091B9
:103EF000C0011091C1012091C2013091C301DC01C8
:103F0000CB0180279127A227B3278093C0019093EC
:103F1000C101A093C201B093C3011F910F910C94F2
:103F2000651B1092BC011092BD011092BE0110924F
:103F3000BF010C94651B41E050E060E070E004C0FC
:103F4000440F551F661F771F8A95D2F74093BC0117
:103F50005093BD016093BE017093BF010C94651B2B
:103F600041E050E060E070E004C0440F551F661F60
:103F7000771F8A95D2F78091BC019091BD01A091E5
:103F8000BE01B091BF01482B592B6A2B7B2B40936C
:103F9000BC015093BD016093BE017093BF010C94AE
:103FA000651B41E050E060E070E004C0440F551F25
:103FB000661F771F8A95D2F740955095609570954A
:103FC0008091BC019091BD01A091BE01B091BF0153
:103FD000482359236A237B234093BC015093BD019E
:103FE0006093BE017093BF010C94651B41E050E0EB
:103FF00060E070E004C0440F551F661F771F8A956C
:10400000D2F78091BC019091BD01A091BE01B09109
:10401000BF01482759276A277B274093BC0150934B
:10402000BD016093BE017093BF010C94651B0F939B
:104030001F930091BC011091BD012091BE013091F0
:10404000BF01DC01CB01802B912BA22BB32B8093E2
:10405000BC019093BD01A093BE01B093BF011F911D
:104060000F910C94651B0F931F930091BC0110914D
:10407000BD012091BE013091BF01DC01CB01802345
:104080009123A223B3238093BC019093BD01A093FD
:10409000BE01B093BF011F910F910C94651B0F934C
:1040A0001F930091BC011091BD012091BE01309180
:1040B000BF01DC01CB0180279127A227B327809382
:1040C000BC019093BD01A093BE01B093BF011F91AD
:1040D0000F910C94651B0895CF92DF92EF92FF929F
:1040E0000F931F93CF93DF938C01C090C001D090AA
:1040F000C101E090C201F090C3014091BC01509118
:10410000BD016091BE017091BF01C42AD52AE62A83
:10411000F72ACFE1D0E0D701C6010C2E04C0B69536
:10412000A795979587950A94D2F780FF07C0B801A5
:104130008C2F0E94940C8130910531F4219758F70F
:10414000B80180E00E94940CDF91CF911F910F91F4
:10415000FF90EF90DF90CF90089590910C019923FC
:1041600021F090910D01911109C020910E01309123
:104170000F01F90132969FEF40E030C0982F9695DD
:10418000969596959F30A0F4E0910E01F0910F0165
:10419000E90FF11D877021E030E0A90102C0440F52
:1041A000551F8A95E2F7CA019181892B8183089571
:1041B0009091D70190FF23C01F928F9389E297E0DF
:1041C0009F938F930E9497080F900F900F900F90DE
:1041D00008959F3F39F04F5F4E3041F05191581391
:1041E000F8CF0DC05111F7CF942FF5CF9F3F39F085
:1041F000F901E90FF11D97FDFA958283089508955D
:1042000090910C01992321F090910D01911109C019
:1042100020910E0130910F01F9013296205F3F4F3E
:1042200030C0982F9695969596959F30A8F4E0917A
:104230000E01F0910F01E90FF11D877021E030E0D0
:10424000A90102C0440F551F8A95E2F7CA01809563
:1042500091818923818308959091D70190FF16C0A1
:104260001F928F938BE097E09F938F930E94970804
:104270000F900F900F900F9008953196E217F3076B
:1042800029F090819813F9CF1082F7CF089581E03B
:1042900090E0E0910E01F0910F01E80FF91F1082FC
:1042A000019680319105A9F708959091D601892B47
:1042B0008093D601089580959091D60189238093AB
:1042C000D60108951092D60108959091D501892BB9
:1042D0008093D501089580959091D501892380938D
:1042E000D50108951092D50108958093C4010895D1
:1042F0001092C401089580910E0190910F01FC016C
:1043000031969C01205F3F4F80E0919191118F5F2A
:10431000E217F307D1F70895E0910E01F0910F0134
:104320008091D6018083E0910E01F0910F01908180
:104330008091D501892B80838091C401882361F00D
:10434000E0910E01F0910F019081892B80830E94F2
:104350007B2181111092C40180910E0190910F0177
:104360000C94A51590933B0180933A010895CF9248
:10437000DF92EF92FF926C01EE24FF24C114D1046E
:10438000E104F10421F0C701B60120E101C020E001
:10439000C72ED82EE92EFF24C114D104E104F10464
:1043A00019F0285FC701B6016B017C0154E0F69457
:1043B000E794D794C7945A95D1F7C114D104E10476
:1043C000F10419F02C5FC701B6016B017C0142E0DA
:1043D000F694E794D794C7944A95D1F7C114D104C1
:1043E000E104F10419F02E5FC701B601DC01CB0135
:1043F000B695A79597958795892B8A2B8B2B09F0D6
:104400002F5F822FFF90EF90DF90CF9008958295DD
:10441000982F9C7C392F36953695282F237344E0AE
:10442000249FC0011124932F982B292F2A7A269597
:10443000892F8575880F822B08951F93CF93DF9363
:104440001F92CDB7DEB799830E940722182F99815A
:10445000892F0E940722212F30E0322F2227A90125
:10446000482BCA010F90DF91CF911F910895809141
:10447000F001843009F11092D80120E488E190E045
:104480000FB6F894A895809360000FBE209360004B
:1044900083B7817F846083BF83B7816083BF789453
:1044A000889583B78E7F83BF88E10FB6F894809399
:1044B0006000109260000FBE089508950895CF9394
:1044C0000E945D220E94390A0E945E22C0E08C2F69
:1044D0000E94650B811104C0CF5FCE30C1F701C0CF
:1044E00081E0CF9108950C94771B82E084BD93E026
:1044F00095BD9AEF97BD80936E0008952FB7F894FD
:104500008091D9019091DA01A091DB01B091DC0199
:104510002FBF0895CF92DF92EF92FF920F931F93D8
:104520002FB7F8944091D9015091DA016091DB01E5
:104530007091DC012FBF6A017B01EE24FF248C0106
:1045400020E030E0C016D106E206F30610F4415038
:1045500051099A01281B390BC9011F910F91FF9036
:10456000EF90DF90CF9008951F920F920FB60F92A9
:1045700011248F939F93AF93BF938091D901909112
:10458000DA01A091DB01B091DC010196A11DB11D02
:104590008093D9019093DA01A093DB01B093DC0101
:1045A000BF91AF919F918F910F900FBE0F901F9071
:1045B00018950E949712F8942FEF87EA91E6215000
:1045C00080409040E1F700C0000087E090EBDC0104
:1045D0008093F9019093FA01A093FB01B093FC0141
:1045E0009CE088E10FB6F894A895809360000FBE18
:1045F00090936000FFCFEF92FF920F931F93CF93A2
:10460000DF93D82FC0E08C2F0E94650B00E010E0F4
:10461000E82EF12CC701002E02C0959587950A94CB
:10462000E2F780FD06C00F5F1F4F0630110591F7BE
:1046300009C0602F7C2F80E00E94720CD813F3CF4A
:1046400081E004C0CF5FCE30F1F680E0DF91CF9102
:104650001F910F91FF90EF900895CF93C82F8CE298
:104660000E94FB22882321F08C2FCF910C94FB22F7
:1046700080E0CF910895CF930E948A24811102C0D7
:104680000E9470248EE497E00E94FE07C5E6C150A8
:1046900049F00E94390A8FE39CE90197F1F700C0C5
:1046A0000000F5CF87E497E00E94FE0789E20E94B0
:1046B0002D23811113C18AE20E942D2381110E94B2
:1046C000702485E00E942D2381110E94D9220E942E
:1046D00095248093D70187E00E942D238823A9F198
:1046E0008BE10E942D23882351F08091D70181FB1B
:1046F000222720F991E0922790FB81F90EC08EE0ED
:104700000E942D23882361F08091D70182FB22270C
:1047100020F991E0922790FB82F98093D70115C090
:1047200080E10E942D239091D701882341F093FBD3
:10473000222720F981E0822780FB93F904C0892F8A
:10474000809580FB90F99093D7018091D7010E94CA
:1047500099240E94A7248093EA0180EE0E942D23D1
:10476000882341F08091EA01982F909590FB80F981
:104770008093EA0189E30E942D23882359F08091D8
:10478000EA0181FB222720F991E0922790FB81F931
:104790008093EA0182EE0E942D23882359F08091B4
:1047A000EA0182FB222720F991E0922790FB82F90F
:1047B0008093EA0186EE0E942D23882359F0809190
:1047C000EA0183FB222720F991E0922790FB83F9ED
:1047D0008093EA0183EE0E942D23882359F0809173
:1047E000EA0184FB222720F991E0922790FB84F9CB
:1047F0008093EA0185E30E942D23882359F080915C
:10480000EA0185FB222720F991E0922790FB85F9A8
:104810008093EA0181E30E942D23882359F080913F
:10482000EA0186FB222720F991E0922790FB86F986
:104830008093EA0181E10E942D23882359F0809121
:10484000EA0187FB222720F991E0922790FB87F964
:104850008093EA018091EA010E94AB248091EA01F1
:1048600087FB882780F980930D0187E20E942D2322
:10487000C82F8EE10E942D238111C2608FE10E941A
:104880002D238111C46080E20E942D238111C86014
:1048900081E20E942D238111C06182E20E942D23BA
:1048A0008111C06283E20E942D238111C06484E2E1
:1048B0000E942D23882311F0C06802C0CC2329F068
:1048C0008C2F0E94A2246C2F03C00E949E24682F6C
:1048D00070E080E090E0CF910C94331FCF91089569
:1048E0006DEE7EEF80E090E00E94732E60E082E04B
:1048F00090E00E94652E60E083E090E00E94652ECB
:1049000060E084E090E00E94652E60E085E090E049
:104910000C94652E80E090E00E945F2E21E08D3E99
:104920009E4F09F020E0822F089582E090E00C94E1
:10493000572E682F82E090E00C94652E83E090E083
:104940000C94572E682F83E090E00C94652E84E041
:1049500090E00C94572E682F84E090E00C94652E24
:104960008091DF0180FF0BC06091130185E0689F9B
:10497000B001112475956795759567952BC081FFDA
:1049800009C06091130185E0689FB00111247595FD
:10499000679520C082FF07C06091130185E0689F82
:1049A000B001112417C09091E0019923D1F06091DA
:1049B0001201961788F72091130185E0289F900136
:1049C0001124929FA001939F500D112470E0CA0101
:1049D0000E94292E6038710540F46115710539F087
:1049E00002C065E070E0862F08958FE7089581E0AA
:1049F00008958091DF0180FF08C06091110170E08F
:104A0000759567957595679521C081FF06C0609182
:104A1000110170E07595679519C082FF04C060911F
:104A2000110170E010C09091E0019923C1F06091F4
:104A300010019617A0F780911101899FC0011124E0
:104A400070E00E94292E6038710528F46115710507
:104A500021F0862F08958FE7089581E0089561E0A1
:104A600070E0F4CF803F21F40E94B024819504C00F
:104A7000813F29F40E94B0248093E3010895823F8E
:104A800021F40E94B024819504C0833F29F40E9440
:104A9000B0248093E2010895893F19F40E94F9241B
:104AA00005C08A3F31F40E94F92481958093E40186
:104AB00008958B3F21F40E94F924819504C08C3F16
:104AC00029F40E94F9248093E5010895843F21F49C
:104AD0008091E101816017C0853F21F48091E1015F
:104AE000826011C0863F21F48091E10184600BC097
:104AF000873F21F48091E101886005C0883F31F44F
:104B00008091E10180618093E10108958D3F21F45E
:104B10008091DF0181600BC08E3F21F48091DF0125
:104B2000826005C08F3F29F48091DF01846080930B
:104B3000DF010895803F39F48091E30187FF6CC065
:104B40001092E30169C0813F29F48091E3011816B6
:104B5000BCF362C09091E201823F29F497FF5CC0F0
:104B60001092E20159C0833F19F41916CCF354C0D6
:104B7000893F41F48091E40118160CF04DC0109269
:104B8000E4014AC08A3F29F48091E40187FF44C0D0
:104B9000F6CF8B3F39F48091E50187FF3DC010923D
:104BA000E5013AC08C3F29F48091E5011816BCF369
:104BB00033C0843F21F48091E1018E7F17C0853F8F
:104BC00021F48091E1018D7F11C0863F21F4809115
:104BD000E1018B7F0BC0873F21F48091E101877F4A
:104BE00005C0883F31F48091E1018F7E8093E1011F
:104BF00013C08D3F21F48091DF018E7F0BC08E3F6B
:104C000021F48091DF018D7F05C08F3F29F48091D1
:104C1000DF018B7F8093DF018091E20181110EC063
:104C20008091E30181110AC08091E401811106C0E5
:104C30008091E501811102C01092E00108958091F8
:104C4000D70183FF7EC08AE897E00E94FE0780912B
:104C5000E1011F928F9385E897E09F938F930E94C5
:104C6000970883E897E00E94FE078091E201282FD1
:104C7000332727FD30953F938F9380E897E09F93EC
:104C80008F930E9497088EE797E00E94FE0780911D
:104C9000E301282F332727FD30953F938F938BE730
:104CA00097E09F938F930E94970889E797E00E946F
:104CB000FE078091E401282F332727FD30953F938D
:104CC0008F9386E797E09F938F930E94970884E7DE
:104CD00097E00E94FE078091E501282F332727FDEA
:104CE00030953F938F9381E797E09F938F930E9436
:104CF00097088EE697E00E94FE078091E0011F92E0
:104D00008F938BE697E09F938F930E94970889E695
:104D100097E00E94FE078091DF011F928F9386E645
:104D200097E09F938F930E94970883E697E00E94F5
:104D3000FE078DB79EB74C960FB6F8949EBF0FBE78
:104D40008DBF81EE91E00E94EE150E947E2290932D
:104D5000DE018093DD0108951F93CF93DF9380914F
:104D6000DD019091DE010E948A22AC019091E00168
:104D7000992321F02091140130E006C02091150103
:104D80008AE0289F900111244217530708F486C037
:104D90008091E201C091E301D091E4011091E5011D
:104DA000811107C0C11176C0D11174C0111172C038
:104DB00075C09F3F19F09F5F9093E001181624F48F
:104DC0000E94B0248093E2018091E20187FF05C038
:104DD0000E94B02481958093E2011C1624F40E9465
:104DE000B0248093E3018091E30187FF05C00E9416
:104DF000B02481958093E3016091E201662339F14B
:104E0000C091E301CC2319F1772767FD7095872FB7
:104E1000972F0E942E2D23E333E343E35FE30E94A9
:104E2000922D0E94FB2C6093E2016C2F772767FD87
:104E30007095872F972F0E942E2D23E333E343E3B2
:104E40005FE30E94922D0E94FB2C6093E3011D16EC
:104E500024F40E94F9248093E4018091E40187FF07
:104E600005C00E94F92481958093E401111624F471
:104E70000E94F9248093E5018091E50187FF05C038
:104E80000E94F92481958093E501DF91CF911F91D4
:104E90000C941F269F3F09F08ECF96CFDF91CF91C4
:104EA0001F910895E1EEF1E085E0DF011D928A9502
:104EB000E9F71092E0011092DF0108958DEA99E080
:104EC0000E94FE071F9281E08F931F9285E08F93CF
:104ED0008FE599E09F938F930E9497080F900F9012
:104EE0000F900F900F900F9008958330E9F128F400
:104EF000813061F0823009F10895853009F462C093
:104F000008F449C0863009F474C0089580911501F1
:104F1000262F30E0280F311D2F3F310524F4680F74
:104F20006093150103C08FEF8093150180911501E7
:104F30001F928F9388E998E072C080911401262F08
:104F400030E0280F311D2F3F310524F4680F6093A6
:104F5000140103C08FEF80931401809114011F92FC
:104F60008F9386E898E05BC080911301262F30E094
:104F7000280F311D2F3F310524F4680F6093130172
:104F800003C08FEF80931301809113011F928F93C1
:104F900083E798E044C080911201262F30E0280F6B
:104FA000311D2F3F310524F4680F6093120103C0B7
:104FB0008FEF80931201809112011F928F938EE5E3
:104FC00098E02DC080911101262F30E0280F311D6F
:104FD0002F3F310524F4680F6093110103C08FEF58
:104FE00080931101809111011F928F9385E498E0C5
:104FF00016C080911001262F30E0280F311D2F3F61
:10500000310524F4680F6093100103C08FEF809383
:105010001001809110011F928F938AE298E09F9374
:105020008F930E9497080F900F900F900F90089504
:10503000833081F128F4813059F08230D1F0089525
:10504000853009F449C0B8F1863009F456C0089596
:1050500080911501681720F4861B8093150102C00A
:1050600010921501809115011F928F938BE198E0AA
:1050700054C080911401681720F4861B809314019A
:1050800002C010921401809114011F928F9389E045
:1050900098E043C080911301681720F4861B809329
:1050A000130102C010921301809113011F928F937C
:1050B00086EF97E032C080911201681720F4861BBA
:1050C0008093120102C010921201809112011F926E
:1050D0008F9381EE97E021C080911101681720F431
:1050E000861B8093110102C0109211018091110161
:1050F0001F928F9388EC97E010C080911001681781
:1051000020F4861B8093100102C010921001809140
:1051100010011F928F938DEA97E09F938F930E94C7
:1051200097080F900F900F900F900895CF93C82F6E
:105130001F928F9382EB9AE09F938F930E94970820
:1051400081E090E0A0E0B0E0BC01CD0104C0660FBA
:10515000771F881F991FCA95D2F70E94331F0F909F
:105160000F900F900F90CF910C94771BCF938D31B0
:1051700009F465C0B0F58E3009F4CCC100F5873074
:1051800009F49BC1A8F4863009F06DC28091D70163
:10519000817F8E7F8093D70187EB9AE00E94FE0784
:1051A00089EF9EE00E94FE0781E08093E70180C1C5
:1051B000883009F44FC08B3009F47CC154C2863169
:1051C00009F4F0C138F4803109F4B8C1813109F42F
:1051D00030C249C2893109F4CEC18B3109F486C18C
:1051E00042C2853309F437C248F4873209F433C226
:1051F00008F433C2893209F42EC235C2833438F43C
:105200008A3308F02CC2883309F454C12CC2833489
:1052100009F421C2883409F026C20E94771B88EE67
:105220009EE00E94FE079FEF23ED80E39150204017
:105230008040E1F700C000000E94D92239C188E017
:105240009FE00E94FE070E94B52C0E9499150E94C3
:10525000CB0D2EC18DEF9EE00E94FE0788EC9CE0F6
:105260000E94FE070E949E241F928F9385EC9CE073
:105270009F938F930E94970883EC9CE00E94FE0707
:105280000E949524C82F80EB9CE00E94FE071F928D
:10529000CF938BEA9CE09F938F930E94970889EAB3
:1052A0009CE00E94FE078FE99CE00E94FE078C2F85
:1052B00081701F928F938CE99CE09F938F930E9443
:1052C00097088AE99CE00E94FE0780E99CE00E9422
:1052D000FE07C1FB882780F91F928F938DE89CE021
:1052E0009F938F930E9497088BE89CE00E94FE0793
:1052F0008FE79CE00E94FE07C2FB882780F91F927F
:105300008F938CE79CE09F938F930E9497088AE786
:105310009CE00E94FE0781E79CE00E94FE07C3FB21
:10532000CC27C0F91F92CF938EE69CE09F938F937A
:105330000E9497088CE69CE00E94FE070E94A7242A
:10534000C82F88E59CE00E94FE071F92CF9383E55B
:105350009CE09F938F930E94970881E59CE00E94B8
:10536000FE0788E39CE00E94FE078C2F81701F924D
:105370008F9385E39CE09F938F930E9497088DB74E
:105380009EB780960FB6F8949EBF0FBE8DBF83E385
:105390009CE00E94FE078CE19CE00E94FE07C1FB9E
:1053A000882780F91F928F9389E19CE09F938F93C8
:1053B0000E94970887E19CE00E94FE0785E09CE040
:1053C0000E94FE07C2FB882780F91F928F9382E01C
:1053D0009CE09F938F930E94970880E09CE00E943E
:1053E000FE078EEE9BE00E94FE07C3FB882780F934
:1053F0001F928F938BEE9BE09F938F930E94970851
:1054000089EE9BE00E94FE078FED9BE00E94FE0765
:10541000C4FB882780F91F928F938CED9BE09F93AC
:105420008F930E9497088AED9BE00E94FE0788EC0C
:105430009BE00E94FE07C5FB882780F91F928F938F
:1054400085EC9BE09F938F930E94970883EC9BE0F1
:105450000E94FE0787EA9BE00E94FE07C6FB8827A2
:1054600080F91F928F9384EA9BE09F938F930E9411
:10547000970882EA9BE00E94FE078AE99BE00E946F
:10548000FE07C7FBCC27C0F91F92CF9387E99BE0AB
:105490009F938F930E94970885E99BE00E94FE07E7
:1054A0008DB79EB74C960FB6F8949EBF0FBE8DBFBA
:1054B000C1E0DEC08EED9AE05BC08091D701C82FBD
:1054C000C17080FF09C08BED9EE00E94FE078091B5
:1054D000D701817F8E7F47C08FEC9EE00E94FE0740
:1054E0008091D70181608093D701E2CF9091D7015D
:1054F00091FBCC27C0F981E0C827892FC0FB81F937
:105500008093D701CC2319F082EC9EE027C084EB76
:105510009EE02EC09091D70192FBCC27C0F981E08C
:10552000C827892FC0FB82F98093D701CC2319F0BB
:1055300085EA9EE013C085E99EE01AC09091D701EC
:1055400093FBCC27C0F981E0C827892FC0FB83F9E2
:105550008093D701CC2351F089E89EE00E94FE079A
:105560008091D70181608093D70182C08CE79EE053
:105570000E94FE079DCF8DE69EE00E94FE0781E41B
:105580009EE00E94FE0784E09EE00E94FE0787EDF9
:105590009DE00E94FE0783E99DE00E94FE0788E6E9
:1055A0009DE0E6CF8AE59DE00E94FE070E949915E6
:1055B0001F928F9380E49DE09F938F930E949708A2
:1055C00080910C011F928F9389E29DE09F938F93AE
:1055D0000E94970880916E011F928F9386E19DE053
:1055E0009F938F930E94970880910D011F928F9334
:1055F00083E09DE09F938F930E9497088091D9014B
:105600009091DA01A091DB01B091DC01BF93AF93DF
:105610009F938F938FEE9CE09F938F930E949708A8
:105620008DB79EB746960FB6F8949EBF0FBE8DBF3E
:105630003FCF0E94771BC0910D0181E0C827C09326
:105640000D01CC2329F085EE9CE00E94FE0710C0DE
:105650008AED9CE08DCF80E003C08D5101C089535D
:105660000E94962825CF88ED9CE00E94FE07C0E0AE
:105670008C2FCF91089580E0089580E00895CF9316
:10568000C82F8091E701813081F020F0823009F449
:105690004FC045C1E0910E01F0910F018081813131
:1056A00069F0823209F03DC109C0E0910E01F0912C
:1056B0000F018081813111F0823261F48C2F0E94C0
:1056C0003B2B811104C08C2F0E94B6282FC081E093
:1056D00090E02CC08C2F0E943D2B811126C0C4313C
:1056E000E1F070F4CB3081F0C031D1F40E945E273C
:1056F0008AEA9AE00E94FE0782E08093E70115C0E3
:10570000C93259F0C83361F487EB9AE00E94FE0772
:105710008EEA9AE00E94FE0708C01092E70103C1DA
:1057200088EA9AE00E94FE07FEC081E08170FDC019
:10573000C43220F5CE3108F0C0C0CB3099F1C8F4A6
:10574000C73009F0D2C08AE08093150194E19093AC
:10575000140193E0909313018093120188E08093E9
:10576000110188E2809310018EE499E00E94FE0707
:10577000BFC0C33149F1C431C1F0B7C0CB3409F463
:10578000A9C028F4C93289F0C83361F0AEC0C13570
:1057900009F49EC0C23509F499C0CE3409F0A5C001
:1057A0006AE09EC00E945E27A3C08091E601882324
:1057B00019F01092E6019CC08BE599E00E94FE076B
:1057C00081E08093E701B1C085E399E00E94FE0784
:1057D00083E299E00E94FE07809115011F928F934A
:1057E00080E299E09F938F930E9497088EE199E061
:1057F0000E94FE078CE099E00E94FE078091140150
:105800001F928F9389E099E09F938F930E9497084E
:1058100087E099E00E94FE0788EF98E00E94FE076B
:10582000809113011F928F9385EF98E09F938F9340
:105830000E94970883EF98E00E94FE0782EE98E0AE
:105840000E94FE07809112011F928F938FED98E0C6
:105850009F938F930E9497088DED98E00E94FE071A
:1058600088EC98E00E94FE07809111011F928F93AF
:1058700085EC98E09F938F930E94970883EC98E0C3
:105880000E94FE078CEA98E00E94FE0780911001BA
:105890001F928F9389EA98E09F938F930E949708B5
:1058A00087EA98E00E94FE078DB79EB748960FB62C
:1058B000F8949EBF0FBE8DBF1BC0CE51EC2FF0E001
:1058C000E15DFE4F80818093E60112C061E003C07C
:1058D00061E006C06AE08091E6010E94752708C079
:1058E0008091E6010E94182803C08CE499E013C05F
:1058F0008091E601882369F01F928F9386E499E0F6
:105900009F938F930E9497080F900F900F900F9086
:1059100004C083E499E00E94FE0781E006C0109273
:10592000E70180E002C080E001CFCF910895E1E877
:10593000F0E08081886080838081816080838FB780
:10594000F89493E09093890090ED909388008FBF36
:105950000895EFE6F0E08081826080830895EFE6AD
:10596000F0E080818D7F80830895EFE6F0E0908104
:1059700082E08927808308951F920F920FB60F92BD
:1059800011242F933F934F935F936F937F938F9344
:105990009F93AF93BF93EF93FF938091E801909112
:1059A000E90101969093E9018093E801811103C018
:1059B00082E00E94CB0DE091E901E695E695F0E0EA
:1059C000E85EF04FE4918091E8018E1303C080E01F
:1059D0000E94CB0DFF91EF91BF91AF919F918F915D
:1059E0007F916F915F914F913F912F910F900FBEDB
:1059F0000F901F90189504D06894B1118DC0089530
:105A000070D088F09F5790F0B92F9927B751A0F028
:105A1000D1F0660F771F881F991F1AF0BA95C9F742
:105A200012C0B13081F077D0B1E0089574C0672F13
:105A3000782F8827B85F39F0B93FCCF386957795F2
:105A40006795B395D9F73EF49095809570956195DB
:105A50007F4F8F4F9F4F0895E89409C097FB3EF406
:105A600090958095709561957F4F8F4F9F4F9923AB
:105A7000A9F0F92F96E9BB279395F6958795779529
:105A80006795B795F111F8CFFAF4BB0F11F460FFE9
:105A90001BC06F5F7F4F8F4F9F4F16C0882311F041
:105AA00096E911C0772321F09EE8872F762F05C055
:105AB000662371F096E8862F70E060E02AF09A95F0
:105AC000660F771F881FDAF7880F9695879597F9E5
:105AD000089557FD9058440F551F59F05F3F71F0DE
:105AE0004795880F97FB991F61F09F3F79F0879545
:105AF0000895121613061406551FF2CF4695F1DFCE
:105B000008C0161617061806991FF1CF869571055D
:105B1000610508940895E894BB2766277727CB0191
:105B200097F908950BD078C069D028F06ED018F09E
:105B3000952309F05AC05FC01124EECFCADFA0F34D
:105B4000959FD1F3950F50E0551F629FF001729F12
:105B5000BB27F00DB11D639FAA27F00DB11DAA1F31
:105B6000649F6627B00DA11D661F829F2227B00D7E
:105B7000A11D621F739FB00DA11D621F839FA00D09
:105B8000611D221F749F3327A00D611D231F849F59
:105B9000600D211D822F762F6A2F11249F575040B0
:105BA0008AF0E1F088234AF0EE0FFF1FBB1F661F4B
:105BB000771F881F91505040A9F79E3F510570F004
:105BC00014C0AACF5F3FECF3983EDCF3869577953F
:105BD0006795B795F795E7959F5FC1F7FE2B880FFF
:105BE000911D9695879597F9089597F99F6780E895
:105BF00070E060E008959FEF80EC089500240A941F
:105C00001616170618060906089500240A94121697
:105C10001306140605060895092E0394000C11F4CA
:105C2000882352F0BB0F40F4BF2B11F460FF04C077
:105C30006F5F7F4F8F4F9F4F0895991B79E004C08E
:105C4000991F961708F0961B881F7A95C9F78095BB
:105C5000089597FB072E16F4009407D077FD09D01E
:105C60000E94432E07FC05D03EF4909581959F4FEE
:105C70000895709561957F4F0895EE0FFF1F059071
:105C8000F491E02D0994AA1BBB1B51E107C0AA1F88
:105C9000BB1FA617B70710F0A61BB70B881F991FCD
:105CA0005A95A9F780959095BC01CD010895F99971
:105CB000FECF92BD81BDF89A992780B50895A8E1DD
:105CC000B0E042E050E00C947A2E262FF999FECFF6
:105CD0001FBA92BD81BD20BD0FB6F894FA9AF99A09
:105CE0000FBE019608950E94652E272F0C94662EF4
:105CF000DC01CB01FC01F999FECF06C0F2BDE1BD8C
:105D0000F89A319600B40D9241505040B8F708957A
:045D1000F894FFCF35
:105D14002002CC0DBD0E9A0E660E320E0101C50195
:105D240028080A03140A3F4D36203998064B0615F5
:105D340006F505BC052F05480561057A059A050198
:0A5D44000203040506070809000029
:00000001FF
